:020000040000FA
:100000006628040000000000622300006223000054
:1000100062230000622300006223000062230000CC
:1000200062230000622300006223000062230000BC
:10003000622300007E230000622300006223000090
:10004000622300006223000062230000622300009C
:1000500062230000EE2500006223000062230000FE
:10006000622300006223000062230000622300007C
:10007000622300006223000062230000622300006C
:10008000622300006223000062230000622300005C
:10009000622300006223000062230000622300004C
:1000A000622300006223000062230000622300003C
:1000B000622300006223000062230000622300002C
:1000C000622300006223000062230000622300001C
:1000D000622300006223000062230000622300000C
:1000E00062230000622300006223000062230000FC
:1000F00062230000622300006223000062230000EC
:1001000062230000622300006223000062230000DB
:1001100062230000622300006223000062230000CB
:1001200062230000622300006223000062230000BB
:1001300062230000622300006223000062230000AB
:10014000622300006223000062230000622300009B
:10015000622300006223000062230000622300008B
:10016000622300006223000062230000622300007B
:10017000622300006223000062230000622300006B
:10018000622300006223000062230000622300005B
:10019000622300006223000062230000622300004B
:1001A000622300006223000062230000622300003B
:1001B000622300006223000062230000622300002B
:1001C000622300006223000062230000622300001B
:1001D000622300006223000062230000622300000B
:1001E00062230000622300006223000062230000FB
:1001F00062230000622300006223000062230000EB
:100200005E280000000000008344550050000000FC
:1002100000277800000006000A0000008444520015
:100220004F5000003E007800000006000A00000069
:1002300084535700414200000080FD00000006008A
:100240000A000000834E4900500000000E87E800BD
:10025000000006000A000000C4545500434B000093
:100260001E27780010079800000006000C00000010
:10027000C4535700415000009E1F7800000F7800C3
:100280004F007800000006000E000000C44F56002A
:1002900045520000002778001E0090000000060074
:1002A0000C000000C3524F0054000000801F780073
:1002B0001E0090003E0F78004F27780000000600D7
:1002C00010000000C4504900434B00000000E9004A
:1002D000000040006E007800000006000E000000E4
:1002E000C4504F004B4500000000E90000004000F2
:1002F0000E0040003E0878003E0078000000060036
:1003000012000000C4524F004C4C00000000E900F5
:100310000C003400811F7800821F78008E0040009E
:1003200081004000911F7800010178000000E90081
:1003300000800900C21078004F0F78004F0178004C
:10034000CF0078003E007800000006002600000084
:10035000C43F4400555000000000B00001003200CE
:1003600000277800000006000E000000823E5200C8
:10037000801F78003E007800000006000A000000A0
:1003800082523E00002778004F00780000000600EF
:100390000A00000082524000002778007FB89700D2
:1003A000000006000A0000008140000010007800F4
:1003B0000000060008000000C24340001040780022
:1003C0000000FB00000006000A000000C121000040
:1003D0003E0878003E007800000006000A00000099
:1003E000C24321001E4878003E0078003E0078009D
:1003F000000006000C000000812B00003E004000C1
:100400000000060008000000C22B2B00811F7800AE
:10041000BE0078003E0040001E8F4800CF007800EC
:100420000000060010000000864E450047415400C1
:10043000450000000000EA00000006000C0000007B
:10044000812D00003E0010000000060008000000A2
:10045000C22D2D00811F7800BE0078003E001000E4
:100460001E8F1800CF00780000000600100000006A
:1004700082322A004100DD00000006000800000072
:1004800082342A004200DD0000000600080000005F
:1004900082322F004180DE000000060008000000CC
:1004A00082342F004280DE000000060008000000B9
:1004B00082303C004F80DE00000006000800000093
:1004C000C2303D000000B000010032000080EF00AB
:1004D0000080EA00000006000E000000C2303E006E
:1004E0000000B000020032000080EA004F80DE0011
:1004F000000006000E000000C2553C003E00100047
:100500000000EF00F2FF3900000006000C000000C0
:10051000C13C00003E0010000000EF00ECFF350081
:10052000000006000C000000C13D00003E00680015
:100530000000EF00E6FF3200000006000C000000A3
:10054000C13E00003E0010000000EF00E0FF3C0054
:10055000000006000C000000C34E4F0054000000D5
:100560000000B000DAFF32000000EF0000000600DB
:100570000E000000C2552A00811F78003E00B8001E
:10058000CF007800000006000C000000C12A000027
:10059000811F78003E80B900CF007800000006007F
:1005A0000C000000C5552F004D4F4400821F7800FD
:1005B000811F7800000178001E00780011000900FA
:1005C0000280D800010F7800CF0078004F0178003A
:1005D000000006001A000000C6552A002F4D4F00EB
:1005E00044000000821F7800811F7800000178001D
:1005F0003E0078001E00B800110009004288D800B3
:10060000010F7800CF0078004F017800000006004D
:100610001E000000C52A2F004D4F4400821F7800A5
:10062000811F7800000178003E0078001E80B9002C
:10063000110009004208D800010F7800CF007800AF
:100640004F017800000006001C000000C42F4D0080
:100650004F440000821F7800811F7800000178005D
:100660001E007800110009000200D800010F780078
:10067000CF0078004F017800000006001A0000004B
:10068000C12F0000811F780080007800F1FF070073
:1006900001F0A300010039008100EA00801F78000A
:1006A0003E00780000F0A300010039000000EA00DD
:1006B0004100DD00810050004F007800CF0078003D
:1006C0000500390000F0A300020031000000E8003E
:1006D000000006000000E9000000060030000000F5
:1006E000C34D4F0044000000DAFF07003E007800D1
:1006F000000006000C000000C22A2F00811F7800B5
:1007000080007800C5FF0700E1FF37000000060009
:100710000E000000C453510052540000831F7800A3
:10072000821F7800811F78000027EB00010820005D
:100730001E8140000211B8000200E10001003900F2
:100740001E8F40008100D100F9FF39001E01E80032
:100750001E11B8000010E100010031001E0FE8007A
:10076000CF0078004F017800CF0178003E0078007C
:100770000000060032000000C34D41005800000098
:100780001E00E10002003C003E0078000000060070
:10079000620747000000060012000000C34D490038
:1007A0004E0000001E00E100F9FF35003E00780019
:1007B000000006000E000000C3414200530000008C
:1007C0000000B00001003B000000EA00000006004D
:1007D0000E00000083414E00440000003E00600017
:1007E000000006000A000000824F52003E00700028
:1007F000000006000800000083584F00520000006F
:100800003E006800000006000A000000C3415300DB
:10081000480000000000B0000800320004003B0067
:100820000080EA00008009001E8FD100030037001D
:100830000000E900008009001E0FD0003E00780093
:10084000000006001E000000C34C530048000000DA
:100850000000B000F9FF3200F5FF3B000080EA0025
:10086000008009001E0FD100F4FF370000000600D1
:1008700016000000C3524F004C0000000000B00002
:10088000EEFF320004003B000080EA000080090017
:100890001E0FD300E9FF37000000E90000800900C7
:1008A0001E0FD200E5FF3700000006001E0000000A
:1008B00083434F004D0000000080EA000000060066
:1008C0000A000000C32B430021000000811F7800B4
:1008D000BE00780010C840003E007800CF007800CD
:1008E0000000060012000000C32D4300210000009C
:1008F000811F7800BE00780010C810003E0078000C
:10090000CF0078000000060012000000C22B21007A
:10091000811F7800BE007800108840003E007800FB
:10092000CF0078000000060010000000C22D21005A
:10093000811F7800BE007800108810003E0078000B
:10094000CF0078000000060010000000C4464900F7
:100950004C4C0000821F7800811F78003E01780017
:10096000BE0078000201E90002800900805878008A
:100970003E007800CF0078004F01780000000600AC
:100980001C000000C5434D004F564500821F7800F3
:10099000811F78003E0178009E001100BE007800A3
:1009A000050039000000E90009003300008009005B
:1009B00031597800060037000201400081004000F4
:1009C0000000E90002003300008009004161780066
:1009D0003E007800CF0078004F017800000006004C
:1009E00030000000C44D4F0056450000821F7800C3
:1009F000811F78003E0178009E001100BE00780043
:100A0000050039000000E9000B00330000800900F8
:100A1000311978000800370002014000020140004F
:100A200081004000810040000000E9000200330026
:100A300000800900412178003E007800CF00780056
:100A40004F01780000000600340000008449440093
:100A50004C4500000140FE00000006000A000000B6
:100A600085534C00454550000040FE000000060044
:100A70000A000000C8535F0054414D00504F4E0023
:100A80000027780000902000000006000E00000003
:100A9000C6535F00574F5200440000000027780003
:100AA00000962000000006000E000000C8535F0002
:100AB000464F52004D41540000277800009A200014
:100AC000000006000E000000C549540052583100D5
:100AD0000027780000A02000000006000C000000A5
:100AE000C55445004C4543000027780040A0200035
:100AF000000006000C000000C6434E00544954009C
:100B0000500000000027780060A0200000000600D0
:100B10000E000000C8534500515545004E434500A6
:100B20000027780080A02000000006000E000000D2
:100B3000C3504100440000000027780020A120009D
:100B4000000006000C000000C33E49004E000000FB
:100B50000027780040A12000000006000C000000E3
:100B6000C94D45004D5F4400455054004800000009
:100B70000027780060A1200000000600100000009F
:100B8000CB4D45004D5F500052474800455245004F
:100B90000027780080A1200000000600100000005F
:100BA000CA414400525F4300524541005445000091
:100BB00000277800C0A120000000060010000000FF
:100BC000C5535400415254000027780000A2200071
:100BD000000006000C000000C55445004D505300B5
:100BE0000027780040A22000000006000C00000052
:100BF000C84D45004D5F480045524500002778002C
:100C000080A22000000006000E000000CA5354001D
:100C10004F505F00464F52005448000000277800B4
:100C2000A0A220000000060010000000C4454F00F4
:100C30004C4E000000277800E0A2200000000600D3
:100C40000C000000C3454F0046000000002778005C
:100C500000A32000000006000C000000C442410078
:100C6000534500000027780020A320000000060064
:100C70000C000000C5535400415445000027780083
:100C800040A32000000006000C000000C5455200F3
:100C9000524F52000027780060A320000000060099
:100CA0000C000000C5495400314D53000027780066
:100CB000C0A32000000006000C000000CA494E003E
:100CC000505554005F4649004C450000002778000D
:100CD00000A420000000060010000000C7505200D1
:100CE000475F50004E5400000027780040AF2000BE
:100CF000000006000E000000C544450050544800A6
:100D000000277800E08F20000E0050004180DE00B8
:100D10000000060010000000C65244004550540078
:100D20004800000000277800408020000080570025
:100D30004180DE000000060012000000C750520093
:100D4000474845005245000091FF07000027780002
:100D5000801F78003E0078002000B000100078006E
:100D6000002778004F00780010007800000006008F
:100D70001C000000C83E5000524748004552450044
:100D800083FF070000277800801F78003E0078006E
:100D90008FFD0700002778004F0078002000B0008A
:100DA0008BFD0700000006001C000000C4454D003C
:100DB0004954000000277800002778003001200007
:100DC000DAFD070033FD070000277800100120003E
:100DD000D6FD07003E007000E1FD07000000B000F6
:100DE0003E0078001E0032003FFF07001000780030
:100DF0000000B0003E0078000E00320000277800AE
:100E000080BB200038FF070071FD07000027780035
:100E1000A0002000C5FD07000000B0003E007800E3
:100E20000300320000277800E002200001003700B4
:100E300000000600002778000000B0003E007800A7
:100E400007003200A1FF07002008B0005BFD07008B
:100E50009CFD07000000B0003E007800F9FF320062
:100E6000002778002022200010007800002778005A
:100E7000002020003E0060000000B0003E0078002E
:100E80000300320000277800000020000500370032
:100E900000277800402220004DFD07000027780041
:100EA000F0FF2F000000B0003E007800ECFF3200A1
:100EB0000000060086000000C450520047400000B9
:100EC00089FF0700811F7800821F7800BE0078002C
:100ED0001000A7001500370002C02F00028160003B
:100EE0001010E10011003A00100190001E10E10006
:100EF0000E003A004000B000E13FB2000080400028
:100F0000C108DE00008040000001EB000000A600E8
:100F1000B0007800304178000000A600B0007800F2
:100F2000020F78000100780005003700220320003E
:100F30001E0978001181BA00020F78001100BA0072
:100F40004F017800CF007800000006004C00000040
:100F5000C45052004721000063FF0700811F780042
:100F6000821F7800BE00780002C02F00028160005E
:100F70001010E10003003A00100190001E10E10083
:100F8000060032001000A6002800070002C02F0053
:100F9000029860001E107800110007004000B000A9
:100FA000E13FB20000804000C108DE000080400048
:100FB00062074700BE0078003E0178000000A600EE
:100FC00001187800025878000000A6000118780087
:100FD0003E0078004F017800CF0078000000060046
:100FE000811F7800821F7800831F7800841F78009B
:100FF000B00078002203200030097800F30F2000B1
:101000001101BA003182BA00021878000458780041
:101010001101BA003182BA00045878000218780031
:101020008301E900F6FF310031003700811F7800AD
:10103000821F7800831F7800841F7800210420001D
:10104000020E2000911F780091087100B000780016
:1010500022042400023B880022032000300978008B
:101060008108BB0052052000323B8800A20A200004
:10107000323B880061E7A80000000000000000008B
:101080007300200012002400023B8800831F7800B8
:10109000F301200030017800304278008208BB0064
:1010A0008498BB0030427800300178008208BB0091
:1010B0008498BB008301E900F6FF3100520520004F
:1010C000323B8800A20A2000323B880061E7A8007A
:1010D000000000000000000061E7AF00FEFF3700E5
:1010E000CF0178008301E900E6FF31004200F900FA
:1010F00041602000008010004F027800CF0178008E
:101100004F017800CF00780000000600E0000000EA
:10111000C4505200472C00000BFF07005DFC070085
:101120005CFC070000277800000020000027780002
:1011300020002000B5FC070011FF070086FF070014
:10114000000006001C000000CB7370005F73790084
:101150006E63700072672100E3FE07001000A600B6
:10116000B2FF07001000A0003E007800000006005B
:1011700032000000C4484500524500009FFE0700B1
:1011800010007800000006000C000000C53E48007A
:101190004552450099FE07008DFC0700000006003F
:1011A0000C000000C2432C00F4FF07000027780069
:1011B0001000B000F7FF07008AFC070000000600DF
:1011C00010000000C12C0000ECFF07000027780091
:1011D0002000B000EFFF07007DFC070000000600C4
:1011E00010000000CA7370005F636F006D706900CB
:1011F0006C65000027FC070026FC070030FF070095
:10120000801F78003E007800002778003E006800CC
:10121000002778007FB8970000277800F0032000AF
:101220003E0060001000B000002778003000200071
:1012300008FD070010FC0700A9FC07003E00100095
:101240004100DD0071FC0700002778004F007800A6
:1012500000277800000420003E0060000000B0007D
:101260003E00780031003200B7FE0700002778000A
:1012700000002000002778002000200063FC070009
:1012800074FC070003FC070000277800F0FF2F0024
:10129000A6FC07000000B0003E0078000D00320000
:1012A000801F78003E0078003E007800002778001C
:1012B00070002000002778004F0078004180DE0099
:1012C00000277800000028003E00700092FF070011
:1012D000150037009CFE0700002778000000200062
:1012E000002778002000200048FC070047FC07008A
:1012F000801F78003E007800002778002000200042
:10130000002778004F00780083FF0700801F7800D7
:101310003E007800002778000000200000277800B9
:101320004F0078007CFF070017003700D9FB07004B
:10133000D8FB0700E2FE070077FF070000277800D0
:101340000000200000277800200020002FFC07006C
:10135000D0FB0700CFFB0700D9FE070059FC0700B0
:10136000C5FB070000277800600020006FFC070025
:101370003E0060000000B0003E007800EBFF32004D
:101380003E0078003E00780000000600E600000005
:101390004249460000277800000B20000027780013
:1013A000000020005CFF0700002778008007200075
:1013B00000277800E003200057FF0700002778008F
:1013C0002003200000277800F0FF2F0052FF0700C5
:1013D0005DFE07000000060026000000C7737000D5
:1013E0005F73610075740000801F78003E00780014
:1013F000801F78003E007800A6FB0700A5FB0700D1
:10140000002778000000200000277800200020003E
:1014100010FC0700AAFE07003E00780000277800B5
:101420004F007800002778004F00780000277800F0
:1014300050002000A5FB0700002778005000200086
:10144000A2FB070003FC0700801F78003E00780025
:1014500000277800F0002000FDFC0700002778003E
:101460004F00780000277800F0FF2F00F8FC0700FD
:101470003E0040000027780040002000A3FB07004A
:101480000027780040002000A0FB0700002778001C
:10149000000020000027780020002000EDFB07005E
:1014A000ADFE0700000006008E00000044454C0021
:1014B00053450000002778007003200000277800C3
:1014C000F0FF2F0014FF07001FFE0700C6FF0700F4
:1014D0001DFE0700000006001800000044544800EC
:1014E000454E000018FE0700BFFF07000000060081
:1014F0000C000000444341005345000000277800E1
:10150000000020000027780000277800000020005D
:1015100000277800601B200036FF0700000006004F
:1015200018000000424F460000277800000020000D
:1015300000277800A01C20002EFF0700002778005D
:1015400000002000002778004029200029FF070024
:1015500090FF0700000006001C00000045454E00FB
:10156000444F4600D3FF0700000006000A000000B9
:1015700047454E004443410053450000E0FD07004D
:101580004180DE0074FB07000000B0003E007800E0
:101590002500320000277800300020004BFB0700B8
:1015A000002778003000200048FB07003E00700054
:1015B0000000B0003E00780008003200801F780074
:1015C0003E007800E0FD070087FF07000027780055
:1015D0004F0078001000B100020037003E00780094
:1015E0003E00780000277800B6FB07000000B0003E
:1015F0003E007800E7FF32003E00780000277800C8
:101600000000200000277800001C2000F9FE0700E1
:10161000002778000000200000277800E01020005C
:10162000F4FE07000200370000277800F0FF2F00CB
:1016300000000600640000004542450047494E0096
:10164000C1FD0700000006000A00000045554E00DD
:1016500054494C004FFF070000277800400020004D
:101660002AFB0700002778004000200027FB070026
:101670005DFF070000000600180000004557480005
:10168000494C450043FF0700000006000A00000027
:1016900046524500504541005400000085FF0700B8
:1016A000002778004000200018FB07000027780082
:1016B0004000200015FB07004BFF0700000006005C
:1016C0001A00000042444F0000277800000020006C
:1016D0000027780080132000C6FE07009AFD07004F
:1016E000002778000000200000277800601B200001
:1016F000C0FE0700002778000000200000277800C7
:10170000601B2000BBFE0700000006002600000052
:10171000452B4C004F4F5000002778000000200060
:1017200000277800001C2000B2FE07000027780088
:101730000000200000277800C01F2000ADFE070039
:10174000002778000000200000277800001C2000FF
:10175000A8FE07000027780000002000002778007E
:1017600060142000A3FE070000277800000020007E
:1017700000277800601420009EFE070000277800F4
:1017800000002000002778008028200099FE070034
:10179000002778000000200000277800C02A2000E1
:1017A00094FE0700ABFF0700002778000000200030
:1017B00000277800E01020008EFE07000027780048
:1017C0000000200000277800E010200089FE0700BC
:1017D0000000060064000000C74C49005445520058
:1017E000414C000000277800800720000027780087
:1017F0000070220048FE070000277800801F780054
:101800003E0078000027780040FF2F0010FC070002
:101810000002B000002778004F0078000027780011
:10182000400020000AFC07003BFE07004AFE0700BC
:101830000000060030000000444C4F004F500000F4
:101840000027780010002000E6FF0700B2FF070025
:101850000000060010000000814900000027780009
:101860007FB89700000006000A000000814A0000CF
:10187000002778005FB89700000006000A0000000B
:10188000814B0000002778003FB897000000060059
:101890000A000000854C45004156450000277800AD
:1018A0004F0078004F007800801F7800801F78007C
:1018B0003E00780000000600140000008445580037
:1018C000495400000000060008000000C243520016
:1018D00000277800D000200036FD070000277800A0
:1018E000A000200033FD07000000060012000000E9
:1018F000C44245004C4C00000027780070002000D6
:101900002CFD0700000006000E000000C55350002B
:1019100041434500002778000002200025FD070014
:10192000000006000E000000C65350004143450071
:101930005300000088FA07000000B0003E00780065
:1019400008003200F3FF07001000B1000027780004
:10195000DCFA07000000B0003E007800F9FF32001A
:101960003E0078000000060022000000C454590028
:101970005045000000277800D9FA07000000B000A9
:101980003E0078002F0032001000B100801F780068
:101990003E0078000027780088FA070000277800CA
:1019A000F00F20003E00600000277800C5FA070015
:1019B00038FA07000027780030002000DBFA070023
:1019C0003E0070000000B0003E00780009003200C8
:1019D0003E007800002778004F0078003E00780035
:1019E0000027780000002000801F78003E0078006B
:1019F0000B0037000027780000277800D000200077
:101A0000CAFA07000000B0003E0078000300320070
:101A10003E007800AEFF070001003700E5FC07003C
:101A20001000B000002778004F00780000277800F1
:101A3000A4FA07000000B0003E007800D2FF320098
:101A400069003700002778004F80DE000000B000FA
:101A50003E00780064003200801F78003E0078006D
:101A60000CFA07000BFA070015FD070000277800A5
:101A70004F0078000000EA00002778000000B00066
:101A80003E00780014003200801F78003E0078008D
:101A90000027780080FF2F006DFB070000277800EB
:101AA00000277800D0002000A0FA07000000B00056
:101AB0003E007800030032003E00780084FF0700FB
:101AC00001003700BBFC0700002778004F007800BA
:101AD0001000B10002003700E7F907003E0078006F
:101AE00000277800801F78003E0078000000B000DA
:101AF0003E007800110032000027780000277800AF
:101B0000D000200089FA07000000B0003E007800F5
:101B1000030032003E0078006DFF0700010037002F
:101B2000A4FC0700002778004F0078001000B100E7
:101B3000801F78003E007800010037003E007800EA
:101B400000277800000020000027780020002000F7
:101B50002EFA0700CFF90700CEF90700D8FC0700DE
:101B6000002778004F007800002778000000B000C0
:101B70003E00780014003200801F78003E0078009C
:101B80000027780000277800F00F20003E0060005A
:101B90000027780000277800D000200063FA0700B3
:101BA0000000B0003E007800030032003E007800E4
:101BB00047FF0700010037007EFC07000027780080
:101BC0004F0078001000B100002778003DFA0700B0
:101BD0000000B0003E007800A7FF32003E00780011
:101BE0003E0078003E0078003E0078003E0078001D
:101BF0000000060046010000C5434F00554E54004A
:101C0000002778001000B0009BF90700EBF90700EF
:101C100000277800F00F20003E0060000000060062
:101C200016000000C92D5400524149004C494E0095
:101C3000470000000027780029FA070000277800F5
:101C400030002000A1F907000027780030002000B4
:101C50009EF907001000B1003E004000D7F90700D0
:101C6000002778000002200030FA07003E006000E4
:101C70000000B0003E007800020032001000B10009
:101C8000ECFF37000000060034000000C3424900AA
:101C90004E0000000027780020002000F1FB070024
:101CA000CBF907000000060010000000C54F4300FC
:101CB00054414C000027780080002000E9FB070019
:101CC000C3F907000000060010000000C7444500EB
:101CD00043494D00414C000000277800A00020003F
:101CE000E0FB0700BAF90700000006001200000040
:101CF000C34845005800000000277800000120007C
:101D0000D8FB0700B2F90700000006001000000031
:101D1000C7434F004E564500525400001000B0001B
:101D200000277800000020005AF90700A3F90700F7
:101D30000027780000277800B0022000FBF9070098
:101D40000000B0003E007800070032003E0078003E
:101D5000801F78003E0078001000B0000027780057
:101D60004F0078000C00370000277800D0022000D8
:101D7000EEF907000000B0003E00780006003200D7
:101D8000801F78003E0078001000B0000027780027
:101D90004F0078001000B100801F78003E007800EE
:101DA0000027780085F907000003B10000277800BC
:101DB0004F80DE000000B0003E00780004003200DA
:101DC0003E00780000277800F0FF2F003500370034
:101DD000002778000027780090002000D9F907003C
:101DE0000000B0003E007800060032007000B10034
:101DF0000027780000277800A0002000C5F9070020
:101E00000200370000277800000020000000B0002A
:101E10003E007800040032003E0078000027780081
:101E2000F0FF2F001F003700002778008DFB070010
:101E300010007800B7F907000000B0003E007800FD
:101E400015003200801F78003E007800801F780067
:101E50003E00780083FB070010007800C6F90700F9
:101E6000002778004F0078001000B00000277800AD
:101E70004F00780000F90700801F78003E007800CE
:101E80003E004000002778004F00780000277800CF
:101E900000002000030037003E0078000027780093
:101EA000F0FF2F000000B0003E007800BCFF3200C1
:101EB000002778004F0078000000B0003E00780056
:101EC00005003200801F78003E0078000000EA0024
:101ED000002778004F00780000000600E8000000AE
:101EE000C23C23000027780000002000F2FA07001F
:101EF0003CF9070000277800801F78003E0078003A
:101F00004F80DE00002778004F0078002CFA070091
:101F1000000006001C000000C4484F004C440000B4
:101F2000E5FA0700002778001000B00000277800CD
:101F30001000B0000027780030002000E3F8070010
:101F40001EF9070000277800F00F20003E00600017
:101F500000277800E005200012FA07008BFA07003E
:101F60000027780015F9070000277800F00F2000FF
:101F70003E0060001000B00000277800E00520005F
:101F800008FA0700C3F8070016F907001000B000B0
:101F900014F907000000060042000000C123000001
:101FA00030FB07001000780080F90700B2F8070046
:101FB0000003B0000027780000277800900320007D
:101FC00060F9070000277800700020003E006000E4
:101FD0003E004000D2FF0700000006002200000083
:101FE000C2235300EEFF0700002778005CF90700CA
:101FF0000000B0003E007800FAFF3200000006004A
:1020000012000000C4534900474E0000A1F8070029
:102010000000B0003E007800030032000027780086
:10202000D0022000BEFF07000000060016000000DE
:10203000C2233E003E0078003E0078009EFA070072
:10204000EFFE0700000006000E000000C12E000099
:10205000A4FF07000027780000022000B0FF07005F
:10206000E0FF0700E9FF0700F2FF070041FE07005D
:102070000000060016000000C13F000010007800BC
:10208000F3FF0700000006000A000000C2552E0002
:10209000002778000000200092FF0700002778004A
:1020A000000220009EFF07003E00780072F8070043
:1020B000CCFF0700DFFF07002EFE07000000060030
:1020C0001C000000C4574F0052440000801F7800DD
:1020D0003E00780071FA0700002778000000200019
:1020E0006CF80700BFF80700002778000000200008
:1020F000D0FA0700B6F8070000277800000020009B
:10210000D2FA0700B2F807008BFA07001000780037
:102110008FFA0700100078003E004000002778008A
:10212000801F78003E0078001000B0000027780083
:102130001000200086FA0700F5F907000027780054
:102140004F0078009DF8070000277800F00F20006E
:102150003E00600000277800801F78003E00780075
:10216000002778003000200058F80700002778008A
:1021700092F807003E0040001000B00099F80700F8
:10218000002778004F00780000277800CDF807007E
:1021900040F807000027780030002000E3F807002F
:1021A0003E0070000000B0003E0078000A003200DF
:1021B0003E00780000277800F0FF2F00002778000D
:1021C0009CFA070082F80700002778009FFA0700B2
:1021D0007FF807002E0037000027780000277800DE
:1021E000D0002000D1F807000000B0003E007800C9
:1021F000070032003E00780000277800F0FF2F0033
:10220000002778008BFA070071F8070020003700DC
:1022100000277800801F78003E00780000277800B3
:1022200090002000C1F80700002778007FB89700D1
:102230000027780000022000BCF807003E00700074
:10224000002778004F007800002778007FB89700BB
:10225000B6F807003E0070000000B0003E007800B5
:102260000300320000277800F0FF2F00080037003D
:1022700000277800100020000027780030002000A0
:1022800012F8070091F907000027780000002000ED
:102290000000B0003E007800A0FF32003E00780051
:1022A000002778004F0078003E007800000006000C
:1022B000F8000000C127000000277800000220007D
:1022C00082FF0700002778003CF807000000B000FC
:1022D0003E007800CE003200801F78003E0078007B
:1022E00039FA070000277800801F78003E00780048
:1022F0002000B00010007800002778004F00780020
:1023000010007800002778007FB897000027780039
:102310000027780029F807003E0040001000B000B8
:102320000027780040002000E8F707000027780029
:1023300040002000E5F70700D6F70700D5F70700B3
:10234000DFFA070000277800F0F32F003E0060005E
:10235000002778004F007800CEF7070000277800AC
:10236000F00F20003E006000CAF7070013F80700D6
:1023700000277800F00F20003E0060006BF8070097
:102380000000B0003E007800350032001000B000C0
:102390000027780060002000CCF70700BDF7070099
:1023A00068F807000000B0003E0078002900320005
:1023B000B8F707000027780080FF2F0024F90700F6
:1023C000B4F70700FDF7070058F807000000B00059
:1023D0003E0078001C0032001000B000002778009A
:1023E00060002000B9F70700AAF7070055F80700BA
:1023F0000000B0003E007800100032000027780096
:1024000030002000B1F70700A2F70700EBF7070044
:1024100046F807000000B0003E00780004003200DB
:102420001000B00000277800F0FF2F0002003700F6
:102430000027780000002000020037000027780005
:10244000F0FF2F0002003700002778000000200076
:102450000200370000277800F0FF2F00020037004D
:102460000027780000002000801F78003E007800E0
:10247000801F78003E0078003E0078003E00780023
:10248000002778004F007800002778004F00780080
:102490000000B0003E0078001F00320000277800E6
:1024A0004000200089F707007AF7070025F80700A9
:1024B0000000B0003E0078000F003200801F78005E
:1024C0003E007800002778000000200000277800F8
:1024D00020002000CDF707006EF707006DF707001A
:1024E00077FA0700002778004F007800002778006F
:1024F00000002000070037003E0078003E00780012
:102500003E0078003E0078003E007800002778000A
:10251000F0FF2F003A0037003E0078003E007800C0
:102520003E007800801F78003E007800801F780011
:102530003E00780057F7070056F70700002778009D
:10254000000020000027780020002000C1F70700CD
:102550005BFA07004FF707004EF707003E007000D8
:102560000000B0003E00780017003200B9F7070005
:10257000002778004F007800002778004F0078008F
:10258000002778004000200050F70700002778005F
:10259000400020004DF707003EF707003DF7070019
:1025A00047FA070000277800F0F32F003E00600094
:1025B000002778006000200044F70700002778001B
:1025C000000020000E003700002778004F00780040
:1025D000002778004F0078003E0078003E00780029
:1025E0003E0078003E0078003E007800002778002A
:1025F0003E0068000027780000277800F0FF2F00D9
:102600000000B0003E00780053FF320003003700A6
:10261000002778003E0068000027780000000600D0
:10262000B8010000C44649004E44000022FF0700E4
:1026300018F7070017F707003E0070000000B00011
:102640003E0078001500320012F7070011F707006E
:102650001BFA0700801F78003E00780000277800F2
:102660003E006800002778004F00780000277800BF
:10267000F00320003E0060001000B000002778004A
:1026800030002000F3F70700FBF6070094F707007F
:102690003E0010004100DD005CF70700000006006E
:1026A00040000000415B000000277800000020008F
:1026B00072F9070046F70700000006000E00000050
:1026C000C15D000000277800F0FF2F006BF90700C4
:1026D0003FF70700000006000E000000C13A0000AE
:1026E000002778000002200078FE070096F9070016
:1026F000002778000000200000277800200020003C
:1027000042F7070030F9070000277800801F7800A3
:102710003E0078002000B00010007800002778000C
:102720007FB89700100078004AF707007AFA070090
:1027300085F90700002778007FB8970024F7070085
:10274000002778004F0078002000B00020F7070035
:102750000027780019F7070000277800F003200011
:102760003E0060001000B000801F78003E0078003E
:10277000002778002000B00010F70700002778003D
:10278000F00F20003E006000C2F607001000B0000D
:102790000AF7070000277800800020002CF80700C7
:1027A000002778007FB897001000B100002778005C
:1027B000000C20003E0070003E00400056FA07006A
:1027C0003000B000002778004F0078003000B100E2
:1027D0000027780042F707000000B0003E007800B4
:1027E00016003200801F78003E0078000027780035
:1027F0002000B000F1F6070000277800F00F20005D
:102800003E006000A3F607001000B000EBF60700E2
:1028100000277800800020000DF8070000277800CE
:1028200030002000A9F60700E4F607000027780032
:10283000F00F20003E006000DFFF37003E00780010
:102840003E00780000277800F0FF2F000BF907000A
:10285000DFF607002AF90700C5F80700DCF60700D5
:1028600000000600C6000000413B00000027780081
:1028700060002000002778000000200026FA0700F2
:1028800035FA07000027780000002000FBF8070059
:10289000CFF607001AF90700B5F807001000780016
:1028A0003E0010000000B0003E0078000E00320034
:1028B0000027780030002000F6F80700C4F6070073
:1028C0009DF8070010007800F2F807002000B00023
:1028D000BFF607009EF8070010007800EDF807002B
:1028E0004000B000BAF607000000060044000000F7
:1028F000C7495400314D53002121000000277800C2
:102900004280BF00801F7800004EB30042E0B70055
:102910003E007800E5F8070000277800801F780067
:102920003E0078002000B000A9F6070000277800DC
:102930004F007800A6F60700002778004F007800C7
:1029400042A0B7003E007800000006003000000002
:10295000C67370005F736500710000000027780087
:102960004F007800002778004F00780049F60700F4
:1029700048F6070047F6070046F6070050F907003B
:102980003E00700074F607000000B0003E007800C2
:1029900013003200801F78003E0078000027780086
:1029A00000002000002778006000200097F6070054
:1029B00038F6070037F6070041F9070000277800CE
:1029C0004F00780082F60700002778003E0068007C
:1029D00000277800200020008CF60700E5FF370074
:1029E0003E0078003E0078004DF807000027780090
:1029F000801F78003E0078006000B00074F6070089
:102A0000002778007FB897004000B00070F60700FC
:102A100000277800F0FF2700002778007FB8970094
:102A20008000B0006AF60700002778000000200050
:102A3000002778007FB897002000B00064F60700F8
:102A4000002778004F00780061F6070000000600BC
:102A5000B20000004A534500515F4200454749001B
:102A60004E5B00000027780000002000002778005F
:102A7000804A2100DFF907000027780000002000CD
:102A80007EF8070052F60700000006001E00000056
:102A9000C7534500515F410044440000E3FE070076
:102AA000FCF50700FBF507003E0070000000B000D9
:102AB0003E0078001100320000277800000020005E
:102AC000AEF9070094F90700002778000000200005
:102AD000BDF9070090F907000027780000002000EA
:102AE000E5F507008CF907000027780000002000BA
:102AF000E1F5070088F90700100037003E00780074
:102B00003E007800002778005000200061F80700A0
:102B10002FF6070008F80700100078005DF807009E
:102B20002000B0002AF6070009F80700100078001E
:102B300058F807004000B00025F607000000060026
:102B40005A000000C8534500515F45004E445D00E7
:102B50000027780000002000002778006EF90700A9
:102B6000D8FE07000000060014000000C5737000C6
:102B70005F2E6700002778004F007800002778005C
:102B80004F007800C3F50700C2F50700CCF8070036
:102B900000277800F00F20003E006000801F7800C2
:102BA0003E0078003E007800BAF50700B9F507004E
:102BB0000027780000002000002778007FB89700E9
:102BC0001000B0000027780030002000A1F60700B8
:102BD000A9F5070042F607003E0010004100DD00A5
:102BE0000AF60700002778004F007800A2F50700DA
:102BF000801F78003E0078009FF50700801F780056
:102C00003E0078000000EA005AFB070000000600C2
:102C100068000000C8534500515F4C004953540000
:102C2000BFF70700002778004000B00010007800D0
:102C300098F507006000B000100078003E007000BA
:102C40000000B0003E007800B600320005F8070032
:102C500010007800801F78003E0078001EFC0700FE
:102C6000C4FF07001050650072696F0064652000A2
:102C700064752000544943003A207500002778000D
:102C80001000780000277800801F78003E00780050
:102C900000277800803E200044F60700ECFC070087
:102CA000002778008000200042F807000027780005
:102CB000C00220003FF807008AFC0700B8FC0700AC
:102CC000B7FC0700B6FC0700DAFC070029FB070089
:102CD000002778003007200036F80700FCFA0700CC
:102CE0004000B00000277800801F78003E00780088
:102CF00010007800002778004F0078002000B00016
:102D00001000780063F5070062F507006CF8070013
:102D10003E0070000000B0003E00780077003200F6
:102D20000027780000002000002778002000200005
:102D3000B6F5070057F5070056F5070060F80700DD
:102D400000277800000020000027780020002000E5
:102D5000C0F507004FF507004EF5070058F80700CB
:102D6000801F78003E0078003E0078000027780041
:102D70004F00780000277800002778000008200026
:102D80003E0060000000B0003E0078000900320004
:102D900000277800F00320003E0060000000EA00F9
:102DA000F4FA0700DBFA070000277800F0FF2F0095
:102DB00002003700002778003E0068000000B000E5
:102DC0003E007800DEFF32006AFF070009706500F0
:102DD00072696F0064653A00207520000027780052
:102DE00000002000002778002000200087F5070061
:102DF00028F5070027F5070031F8070000277800BD
:102E00007FB8970000277800803E2000F5F5070086
:102E10008FFC07000027780080002000E5F70700FE
:102E200000277800C0022000E2F707002DFC070011
:102E30005BFC07005AFC070059FC07007DFC0700FB
:102E4000CCFA07003E007800002778003007200009
:102E5000D8F7070047FF070009207200657461007A
:102E600072643A00207520000027780000002000DE
:102E7000002778002000200064F5070005F5070012
:102E800004F507000EF80700002778007FB89700C8
:102E900000277800803E2000D2F507006CFC070078
:102EA0000027780080002000C2F707000027780084
:102EB000C0022000BFF707000AFC070038FC07002B
:102EC00037FC070036FC07005AFC0700A9FA070088
:102ED0003E0078000027780030072000B5F7070093
:102EE0000027780000002000002778002000200044
:102EF00046F5070076FA070082FF37003E007800AB
:102F00003E007800002778004F0078003E007800EF
:102F1000002778004F00780052F707002CF50700D3
:102F2000090037003E00780012FF070010415500ED
:102F300043554E004520530045515500454E430032
:102F4000452E750062FA0700000006009E01000091
:102F500047434F004D5049004C450000D6FC070048
:102F6000CCF40700CBF407003E0070000000B00076
:102F70003E00780009003200BFF4070019FA07008C
:102F800018FA0700002778000000200000277800CA
:102F9000208F200097F80700100037003E007800CF
:102FA0003E007800002778003000200039F7070045
:102FB00007F50700E0F607001000780035F7070076
:102FC0002000B00002F50700E1F6070010007800CD
:102FD00030F707004000B000FDF4070000000600D5
:102FE0004A000000495B43004F4D5000494C4500EA
:102FF0005D000000B0FC0700A6F40700A5F4070080
:103000003E0070000000B0003E0078000200320078
:1030100078F80700100037003E0078003E00780086
:1030200000277800300020001AF70700E8F40700B6
:10303000C1F607001000780016F707002000B00066
:10304000E3F40700C2F607001000780011F707004C
:103050004000B000DEF40700000006003E00000063
:10306000C74558004543550054450000801F78006F
:103070003E007800801F78003E00780000000600C7
:1030800012000000C122000000277800400020004C
:10309000FAF607001EF607002BF707000027780056
:1030A000F00F20000027780000002000000006003C
:1030B00018000000422E22000027780000002000A7
:1030C00000277800605B21004AF80700EEFF070048
:1030D0000000060012000000012800000027780010
:1030E00020002000E5F6070009F6070000000600B2
:1030F0000E000000C22E530001F7070096F40700EF
:103100000000B0003E0078001C003200002778006C
:1031100000002000801F78003E0078000027780023
:103120001000B000002778007FB897003E00100024
:1031300066F40700C6FB0700002778004F00780000
:103140001000B00000277800801F78003E00780053
:1031500050F40700EFF4070001F507000000B0008D
:103160003E007800EDFF3200002778004F00780025
:103170003E0078003E007800060037007DFE070024
:103180000C5069006C6520007669640065202100A0
:10319000204E4300000006005400000049494D0045
:1031A0004D454400494154004500000086F60700A3
:1031B00000277800801F78003E0078002000B000D3
:1031C00010007800002778004F0078001000780089
:1031D00030F407002FF4070039F7070000277800C4
:1031E000F0F72F003E00600000277800400020002C
:1031F00046F40700002778004000200043F4070051
:1032000055F707000000060038000000464449005A
:1032100052454300540000006BF607000027780079
:10322000801F78003E0078002000B0001000780079
:10323000002778004F0078001000780015F4070090
:1032400014F407001EF7070000277800F0FB2F009A
:103250003E00600000277800400020002BF40700AB
:10326000002778004000200028F407003AF7070004
:103270000000060036000000C5414C004C4F5400D1
:10328000002778000000B0003E0078000500320002
:103290000027780000002000CBF707001000B100E5
:1032A000F7FF37003E007800000006001C00000019
:1032B000C44C4F004144000076F60700100078002F
:1032C0000000B0003E007800020032003E007800AE
:1032D000E901370018F6070010007800801F780019
:1032E0003E0078001AF6070010007800801F780072
:1032F0003E0078004FF6070010007800801F78002D
:103300003E00780051F6070010007800801F78001A
:103310003E00780008F607002DF40700002778002B
:10332000000020000AF6070029F4070053F6070002
:10333000100078000027780069F407000000B00052
:103340003E007800B6003200002778002000200000
:103350007CF407000000B0003E007800A1003200BD
:10336000002778002002200058FB070024FA0700FD
:103370000027780030002000D4F3070000277800F1
:10338000F00F20005DF40700C2F3070054F40700BB
:103390003E0060000000B0003E0078002C003200CB
:1033A000801F78003E007800801F78003E00780083
:1033B000B1F30700E8F307000000B0003E0078001A
:1033C0001700320000277800002778000010200046
:1033D0004AF407000000B0003E0078000800320008
:1033E000002778007FB89700F4F3070000277800E3
:1033F0008000200016F507003E004000070037005F
:10340000002778007FB89700ECF307009AF30700D5
:1034100041F7070000277800000020000300370074
:10342000002778007FB89700E4F3070092F30700C5
:103430001000B000002778004F0078001000B000A6
:10344000002778004F0078001000B100C8FF370057
:103450003E007800D9F307000027780000277800A5
:103460002002200031F407000000B0003E00780088
:103470002A0032003E007800801F78003E0078006D
:10348000B5F307000000B0003E00780004003200F1
:10349000002778000000200077F307001EF70700E0
:1034A0007CF307007BF3070085F607000027780010
:1034B00000F02F003E006000002778004F007800E9
:1034C0003E00400000277800400020007FF3070006
:1034D00000277800400020007CF307009EF60700DC
:1034E000E6F5070010007800002778003000200083
:1034F0000EF407000000B0003E0078000200320029
:103500003E0078003E007800002778004000200050
:10351000DAF5070006F5070031003700CBF50700A4
:10352000100078000000B0003E0078000300320078
:103530003E00780000277800D000200055F30700F7
:1035400000277800F00F2000ECF307000000B00027
:103550003E00780021003200801F78003E00780095
:1035600045F307007CF307000000B0003E00780040
:103570001500320000277800002778000010200096
:10358000DEF307000000B0003E00780007003200C4
:10359000002778004F007800002778008000200086
:1035A000ABF407003E00400006003700002778001B
:1035B0004F00780030F30700D7F6070000277800A7
:1035C0000000200002003700002778004F0078003C
:1035D00029F307001000B000010037003E0078001A
:1035E0000E0037000027780000022000B7FA07001D
:1035F000100078000027780010902200CBF307001D
:103600000000B0003E00780004003200002778007F
:103610002000200099F50700C5F40700EB003700F3
:103620003E00780024FB07001AF3070019F3070097
:103630003E0070000000B0003E0078005F003200E5
:103640008EF50700100078000000B0003E00780002
:10365000240032000FF307000EF3070018F60700EE
:1036600005F307003E0078000027780000082000DE
:103670003E0060000000B0003E0078000200320012
:10368000DCF607001600370002F3070001F307001D
:103690000BF60700801F78003E00780000277800B6
:1036A0003E006800002778004F007800002778006F
:1036B000F00320003E0060001000B00000277800FA
:1036C00030002000E3F30700EBF2070084F307006B
:1036D0003E0010004100DD004CF3070063FE0700D0
:1036E00035003700EBF20700EAF20700F4F50700B7
:1036F000E1F207003E00780000277800000C20006F
:103700003E006000002778000004200087F30700D7
:103710000000B0003E007800110032003E0078004A
:103720003E007800002778002000200059F50700AF
:1037300027F3070000F507001000780055F5070093
:103740002000B00022F3070001F507001000780008
:1037500050F507004000B0001DF3070016003700C9
:10376000CCF20700CBF20700D5F50700801F7800E8
:103770003E007800002778003E00680000277800AF
:103780004F00780000277800F00320003E00600022
:103790001000B0000027780030002000ADF30700D3
:1037A000B5F207004EF307003E0010004100DD00B7
:1037B00016F307002DFE0700840037003E00780056
:1037C000B6F4070000277800FCF207000000B00004
:1037D0003E0078007B003200AEF20700ADF2070039
:1037E0004EF90700B1F207003E007800AFF2070083
:1037F0003E00780000277800F0F2070000277800EC
:103800001002200043F307000000B0003E007800E3
:10381000080032003E00780018F50700100078001C
:103820000000B0003E00780001003200EDF7070014
:103830006300370000277800E0F2070000277800D7
:1038400000277800B002200038F307008AF2070052
:1038500000277800D002200034F307003E007000FB
:103860008CF207001000B000D4F2070000277800A7
:103870001002200027F307003E0060000000B000A7
:103880003E0078003E00320082F207000000B000E7
:103890003E00780037003200C8F20700F7F4070056
:1038A000100078000000B0003E00780027003200D1
:1038B000801F78003E0078000027780000277800FD
:1038C000004020000DF307000000B0003E0078002B
:1038D0000E0032000027780040002000DCF30700D3
:1038E000002778004F00780000277800D0022000E1
:1038F0000EF3070000277800100020003E00600053
:10390000000BB0005CF207000E003700B5F70700AF
:103910000027780000042000002778004F0078007E
:1039200000277800D002200000F30700002778006D
:10393000000320003E0060003E00100000277800D9
:10394000E0032000F4F507000900370000277800A5
:10395000B0022000F5F207000000B0003E00780041
:10396000020032003E004000010037003E0010001F
:10397000020037003E0078003E007800100037005B
:103980003E0078003E0078000027780010002000FC
:10399000C0F407008EF2070067F4070010007800FB
:1039A000BCF407002000B00089F2070068F40700AB
:1039B00010007800B7F407004000B00084F2070060
:1039C000020037003E0078003E0078009FF40700B8
:1039D00010007800AFF40700100078003E0070007F
:1039E0000000B0003E00780050FE3200C4F4070032
:1039F0004F80DE000000B0003E0078000E00320074
:103A00000027780040002000A2F4070070F20700B1
:103A100049F40700100078009EF407002000B00071
:103A20006BF207004AF407001000780099F40700D1
:103A30004000B00066F20700002778004F007800D1
:103A400082F4070062F20700002778004F00780038
:103A500078F407005EF20700002778004F00780036
:103A60003BF407005AF20700002778004F00780067
:103A700031F4070056F2070000000600E8030000DA
:103A8000C64352004541540045000000BBF5070005
:103A900054F70700ACF4070045F40700002778004E
:103AA000801F78003E00780049F207000027780068
:103AB0004F0078002000B00045F207000027780092
:103AC0004000200000277800F0FF2F0092F507004B
:103AD000002778000000200000277800F007200071
:103AE0008DF507009CF50700000006003800000077
:103AF000C87370005F646F0065733E002CF40700AC
:103B000000277800801F78003E0078002000B00079
:103B100010007800002778004F007800100078002F
:103B20000027780000002000002778004F00780070
:103B30000027780040002000E4F10700002778000B
:103B400040002000E1F1070000277800000020007D
:103B500000277800200020002CF20700FEF4070068
:103B60000027780040002000002778004F007800F0
:103B70000027780040002000E4F1070000277800CB
:103B800040002000E1F10700F3F4070072F50700A0
:103B9000002778000000200038F407000CF207002E
:103BA000000006009400000045444F0045533E00CD
:103BB00000277800000020000027780080D721002F
:103BC0008CF507000000060012000000C8564100F6
:103BD00052494100424C4500C1FA0700ABFF0700C3
:103BE00079F50700C5FF070000000600120000007D
:103BF000C8434F004E535400414E5400B8FA0700DA
:103C0000F8F6070000277800600020000027780001
:103C10000000200040F507004FF50700002778005E
:103C20000000200015F40700E9F10700000006007D
:103C300022000000C653540052494E0047000000C5
:103C4000A7FA07008CF10700E6F60700E5F6070083
:103C50000027780060002000002778000000200086
:103C60002DF507003CF50700002778000000200034
:103C700002F40700D6F1070000000600260000004D
:103C8000C5564C0049535400CFF307000027780075
:103C9000801F78003E0078002000B00010007800FF
:103CA000002778004F0078001000780079F10700B5
:103CB00078F1070077F1070076F1070080F407003C
:103CC000801F78003E0078003E00780000277800D2
:103CD0004F00780000277800F00320003E006000CD
:103CE0000000EA0023F707000AF7070069F1070060
:103CF00068F1070000277800000020000027780006
:103D000020002000D3F107006DF4070061F10700E7
:103D100060F107003E0070000000B0003E00780037
:103D200004003200CBF107000027780000002000DB
:103D3000040037003E0078003E007800002778003D
:103D4000F0FF2F000000B0003E007800D7FF3200E7
:103D50003E0078003E007800000006007000000081
:103D6000C34B450059000000D8F307000027780036
:103D70001000B00091F107000140FE0045F107007E
:103D80008EF1070043F107003E0010000000B00074
:103D90003E007800F8FF32003EF107003E00400090
:103DA0002000B00085F10700801F78003E007800F9
:103DB0001000B0000027780080F107001000B0006C
:103DC00000277800F00720003E0060002AF107007D
:103DD00084F10700002778004F00780000000600FB
:103DE00042000000C5494E004B455900B7F307009B
:103DF0000027780071F1070000277800002778007D
:103E00003000200031F107001000B00075F107000C
:103E10001000B10000277800F00720003E0060008D
:103E20003E0040002000B00064F1070000000600E2
:103E300028000000C84B450059424F004152440041
:103E4000A2F307001000B000002778001000B100B6
:103E50005AF107000FF1070058F107003E0010006B
:103E60000000B0003E007800060032000027780015
:103E700052F107003E0040001000B0004FF1070073
:103E800002003700002778003E00680000000600AE
:103E900030000000C6455800504543005400000063
:103EA00000277800F00F20003E0060000027780017
:103EB00000002000002778003000200003F10700F8
:103EC00048F10700F3F007001000B000F1F0070020
:103ED00000277800000220009EF20700A2FF0700E2
:103EE0000027780000277800F001200095F10700F6
:103EF000E8F0070000277800F007200085F10700B0
:103F00003E006000E3F007000027780090002000EA
:103F100086F107003E007000002778004000200076
:103F2000EAF0070025F10700002778004000200094
:103F3000E6F0070077F107003E0060000000B000E7
:103F40003E00780047003200002778000027780004
:103F50009000200075F107000000B0003E007800DE
:103F6000180032003E007800002778000002200090
:103F70000027780080002000002778004000200003
:103F8000D2F007000DF1070000277800801F7800AD
:103F90003E00780000277800700020003E0060009E
:103FA0003E0010000027780030002000C7F0070016
:103FB000002778004F0078003E001000F9F107005C
:103FC000020037000027780010002000801F7800D2
:103FD0003E00780000277800801F78003E007800BF
:103FE0000027780073F307000027780030002000D6
:103FF000B6F00700F1F007001000B00000277800CD
:1040000040002000B1F00700F6F00700002778001C
:1040100030002000ADF0070000277800E7F007002F
:104020003E004000EFF00700002778004F007800C6
:10403000002778004F0078001000B10000277800BA
:1040400020F107000000B0003E007800DFFF3200E2
:104050003E0078003E007800002778000000200035
:104060004F0037000027780000277800F007200075
:104070002EF1070087F0070000277800800020005D
:104080002AF107003E00700082F007000027780048
:10409000C001200025F107003E00700000277800D5
:1040A0004000200089F00700C4F007000CF1070071
:1040B0003E0060000000B0003E00780014003200B6
:1040C0003E00780073F00700BCF00700002778007E
:1040D000100020003E001000002778003000200073
:1040E0007AF00700BFF0070000277800800020006A
:1040F00030F3070007F60700002778008000200053
:104100002CF307000027780000002000240037006F
:1041100000277800002778003000200003F1070016
:104120005CF0070000277800D0002000FFF00700B7
:104130003E00700057F00700E2F007003E007000FC
:104140000000B0003E0078000B003200002778002D
:10415000300020005DF007000027780097F007008E
:104160001000B0003E0040009EF0070000277800DD
:10417000F0FF2F000A00370000277800A000200081
:10418000EAF00700F6F007000000B0003E007800FB
:1041900001003200D8F50700002778000000200059
:1041A0000000B0003E0078004CFF32003E00780076
:1041B0003E0078000000060094010000C451550044
:1041C000495400000F8020000027780000002000E4
:1041D00000277800A9F207007DF00700ADF2070084
:1041E0007BF00700A5F20700100078005AF00700E6
:1041F0000000B0003E007800150032000027780073
:104200004F80DE000000B0003E0078000400320065
:104210003E00780000277800A00320000B00370044
:104220000027780020002000C6F007000000B00042
:104230003E007800030032000027780020022000B2
:1042400002003700002778008002200002003700BB
:1042500000277800E0032000D6F2070008F20700EC
:104260000027780020F20700100078000000B0005E
:104270003E0078000300320000277800F00520009F
:104280000200370000277800E004200004FF070048
:104290008FF507000027780030002000FDEF0700B1
:1042A0000027780045F007003E0040001000B000F5
:1042B0004CF007000027780000002000F5EF070011
:1042C00048F007001000B00007F207001000780067
:1042D0000000B0003E00780008003200002778009F
:1042E00030012000B3F20700F3FB0700002778003D
:1042F00010012000AFF2070001003700EEFB0700BD
:1043000064F20700100078000000B0003E00780062
:10431000B50032000E902000F3F107001000780085
:104320000000B0003E00780009003200C4FE070023
:104330000000B0003E007800020032008AFE070054
:104340003E007800002778000000200002003700BF
:1043500000277800F0FF2F000000B0003E0078003A
:10436000EDFF320045F207001000780000277800CA
:10437000F0FF2F006DF007000000B0003E00780055
:104380002000320010F2070000277800801F78001C
:104390003E0078002000B000100078000027780070
:1043A0007FB8970010007800BAEF0700B9EF070058
:1043B000B8EF0700B7EF07000027780000002000E3
:1043C000002778002000200022F00700BCF2070040
:1043D00020F00700002778007FB89700FCEF070067
:1043E000002778004F0078002000B000F8EF0700A9
:1043F00063F2070000277800000020001FF207008A
:10440000F3EF0700DBF90700052A2A002A2A20001B
:10441000A2F10700FAF5070056F507003DF5070081
:104420001CF20700100078000027780000277800B1
:10443000100020003DF007000000B0003E007800B2
:104440000A003200CBF90700183A2000496E7300C9
:1044500074727500637469006F6E2000494E4300EA
:104460004F4E4E00554520002174780000277800FB
:1044700000277800200020002CF007000000B0008A
:104480003E0078000A003200BAF90700193A20000D
:10449000496E730074727500637469006F6E20005A
:1044A000494D4D00454449004154450020217800C4
:1044B0000027780000277800300020001BF007005C
:1044C0000000B0003E0078000B003200A9F90700A0
:1044D0001B3A200050524F00424C45004D452000F1
:1044E00050696C00652064006520520045544F00FF
:1044F00055522000210D5400002778000027780035
:104500004000200009F007000000B0003E007800E5
:104510000B00320097F907001D3A200050524F005F
:10452000424C45004D45200050696C0065206400F8
:1045300065732000444F4E004E4545005320210036
:10454000002778000027780050002000F7EF0700D0
:104550000000B0003E0078000E00320085F9070030
:1045600024494D00504F5300534942004C45200010
:10457000642769006E7365007265720020636500D0
:104580007474650020534500515545004E43450065
:10459000215F63000027780000277800500020008A
:1045A000E8EF07000000B0003E007800080032008D
:1045B00070F907000C3A2000455252004555520050
:1045C000206E6F0020276900A1F607000100370068
:1045D0003E007800C8F40700BDF40700002778000B
:1045E000F0FF2F000F003700A4F107001000780043
:1045F000B4EF07000000B0003E0078000700320072
:1046000000277800F0042000EAF107000027780076
:10461000B0042000E7F10700ADF4070000277800A0
:10462000000020000000B0003E007800EDFE3200E7
:1046300000277800000020000000B0003E00780055
:10464000E0FE32000000060048020000C5414200C2
:104650004F5254000E902000BFF207000027780050
:10466000000020000027780033F1070058EF070012
:1046700037F1070056EF070095F407003DF90700F2
:10468000262A2A002A2A2000494E54004552520068
:1046900055505400494F4E00204C6F00676963002D
:1046A00069656C006C652000284142004F5254003F
:1046B0002920210086F407008FF40700C1FE0700BF
:1046C0000000060000277800600320000027780023
:1046D000801F78003E0078001000780000277800E6
:1046E0004F007800002778001000200005F1070037
:1046F00087F0070036EF070000400600002778002B
:104700006003200000277800801F78003E007800BA
:1047100010007800002778004F007800002778000C
:10472000100020002EF1070079F007000027780024
:104730004008200000277800801F78003E007800A5
:10474000100078000027780070FF2F003E00600006
:10475000002778004F0078001DEF0700E2F0070007
:10476000100078000000B0003E0078002C003200FD
:10477000DDF0070000277800801F78003E007800F9
:10478000100078001000B1000027780000277800A2
:104790004F0078000EEF07004AEF07000000B0005E
:1047A0003E0078001E00320048F107000027780024
:1047B00002EF07001000B00000277800F00720008B
:1047C0003E006000B3EE07001000B000FBEE0700F3
:1047D000B0EE070055EF07000000B0003E00780083
:1047E000030032003E0078003E0078000C003700E5
:1047F00000277800D000200000277800300020003B
:10480000B2EE070000277800ECEE07003E00400003
:104810002000B000F3EE070097EE0700F1EE07006E
:1048200022F1070000277800801F78003E00780002
:1048300010007800002778004F0078002000B000BA
:104840001000780093EE070092EE07003E00700023
:104850000000B0003E0078000200320003FA0700BA
:10486000020037003E0078003E007800ACF0070000
:10487000002778008000B000100078001000B00021
:104880004F80DE000000B0003E00780037003200AC
:10489000E2F0070000277800801F78003E007800D3
:1048A00010007800002778004F0078002000B0004A
:1048B0001000780077EE070076EE07003E007000EB
:1048C0000000B0003E00780026003200002778008B
:1048D0000000200000277800D0F0070000277800B3
:1048E000801F78003E007800B9EE070000277800AE
:1048F0004F0078002000B000B5EE07008EF00700F2
:10490000100078000000B0003E0078001200320075
:1049100000277800F00720003E00600000277800A4
:104920004F0078000027780000F82F003E0060005C
:104930003E004000002778004F0078003E007800DD
:104940004DEE0700801F78003E007800801F780041
:104950003E007800020037003E0078003E007800FC
:10496000020037003E0078003E0078000027780003
:10497000100078000000B0003E0078009400320083
:10498000002778002000B000100078001000B1006F
:10499000002778004F80DE000000B0003E00780065
:1049A000880032003BEE0700100078003E00400017
:1049B00038EE07002000B00085EE070000277800E1
:1049C0000000200033EE07004000B0000027780010
:1049D000801F78003E0078001000780000277800E3
:1049E0004F0078002000B0001000780029EE07008A
:1049F00028EE070032F107003E00700056EE070077
:104A00000000B0003E0078006A003200801F78008D
:104A10003E007800801F78003E007800801F7800FC
:104A20003E0078001000B000002778004F007800AA
:104A3000002778004F007800002778007FB89700A3
:104A4000100078001000B100002778004F80DE00D1
:104A50000000B0003E0078004D00320000277800D2
:104A60005000200019EE07008000B0001000780010
:104A7000002778005000200014EE0700B1EE070078
:104A80000000B0003E0078003D003200801F78003A
:104A90003E007800FFED0700FEED070000277800DC
:104AA00000002000002778004000200057EE07009B
:104AB00003F10700002778004F0078003E00400017
:104AC000002778004F00780041EE07003E00780094
:104AD0000027780040002000FCED07008000B000B7
:104AE00000277800801F78003E00780010007800D2
:104AF0000027780040002000F4ED07000027780030
:104B00004F00780032EE07000027780030002000C8
:104B1000EEED07000027780030002000EBED0700E5
:104B200000277800000020000027780020002000E7
:104B300036EE0700E2F00700002778004280BF0051
:104B4000801F78005FF89700004EB20042E0B70087
:104B50003E00780045F90700002778004F007800F4
:104B600042A0B7003E0078000027780050002000E7
:104B7000D6ED07008000B00015EE070003003700F7
:104B8000002778004F00780011EE0700030037007F
:104B9000002778004F0078000DEE0700002778000E
:104BA00000002000002778008000200017EE07009A
:104BB0008EFF37003E0078003E0078003E0078000F
:104BC00003003700B3ED07002000B00000EE07003F
:104BD0003E007800FEED0700004006000027780048
:104BE0006003200000277800801F78003E007800D6
:104BF00010007800002778004F0078000027780028
:104C000060222000EDED070000277800400820001A
:104C100000277800801F78003E00780010007800A0
:104C200000277800F07F2F003E006000002778000A
:104C30004F007800E6ED0700A5EF07000027780099
:104C4000801F78003E0078002000B000100078003F
:104C5000002778004F007800100078008DED0700E5
:104C60008CED07003E0070000000B0003E007800B0
:104C700002003200FDF80700460037003E007800D1
:104C80003E007800002778001000B1000000B0005E
:104C90003E007800320032000027780000277800BC
:104CA0003001200021EE07007AED07000027780090
:104CB000100120001DEE07003E0070000000B00053
:104CC0003E00780007003200002778003001200005
:104CD00016EE0700FDEF07002008B000C1ED070049
:104CE0001E003700F9EF070000277800B3ED07003A
:104CF0001000B00000277800F00720003E006000A0
:104D000064ED07001000B000ACED070061ED070096
:104D100006EE07000000B0003E00780004003200FC
:104D20003E0078003E0078003E0078000B0037001F
:104D30005EED0700002778003000200063ED0700DB
:104D4000002778009DED07003E0040002000B000E5
:104D5000A4ED070048ED0700A2ED07000D003700A5
:104D6000002778003E0068000027780060322200AB
:104D7000AAEF070000277800801F78003E00780027
:104D800093ED0700002778004F0078002000B00066
:104D90008FED07008EED070000400600AA0300001B
:104DA000D15449004D455200315F550041525400E5
:104DB000315F49004E49540000277800000220006E
:104DC000002778004074200081ED0700002778005C
:104DD000F0CF270000277800201020007CED07008E
:104DE00000277800000028000027780040102000ED
:104DF00077ED0700002778004004200000277800A6
:104E00008022200072ED07000027780000002000BB
:104E1000AEEF07006EED0700002778008000280045
:104E2000002778000022200069ED070000277800A5
:104E300000402000002778002022200064ED0700B9
:104E4000002778008080200000277800400920009B
:104E50005FED0700002778000000200029EF070021
:104E60005BED07000000060066000000C554450029
:104E70004D504F005AEF0700100078000140FE002F
:104E800004ED070056EF07001000780000277800B7
:104E9000300020000DED07003E00100097ED0700E8
:104EA0000000B0003E007800F4FF32003E007800C1
:104EB0003E0078000000060028000000C5464F00B4
:104EC000525448002BF70700CC0D45006E74720059
:104ED000657A200064616E0073206C0065206D00AF
:104EE0006F6E640065206400752046004F525400C8
:104EF000480D0D0020202000202043006F70790015
:104F000072696700687420006A7062002E666F0024
:104F1000727468000D0D4E006F79610075205300AA
:104F200045515500454E43004555520020706F00D5
:104F30007572200050494300323446004A0D20006B
:104F40005665720073696F006E2031002E3030009C
:104F50002020640075203200322F3000352F3200BF
:104F6000303136000D20200068747400703A2F0034
:104F70002F6A7000622E66006F727400682E6600E1
:104F8000726565002E6672002F0D2000206A700089
:104F9000625F66006F7274006840790061686F003C
:104FA0006F6772006F757000732E63006F6D0D0078
:104FB0000D205100756520006C652000464F5200A1
:104FC00054482000736F69007420610076656300A7
:104FD00020544F0049210D000D696E0000000600AD
:104FE00094000000C6464F005247450054000000A0
:104FF000B1F40700A7EC0700A6EC07003E00700024
:105000000000B0003E0078001D003200A1EC070057
:10501000A0EC07000027780000002000002778009F
:10502000200020000BED07009AEC070099EC070028
:1050300053EF0700A2EF070006ED0700E2EE0700BE
:1050400000277800801F78003E007800E0EC070021
:10505000002778004F0078002000B000DCEC07004B
:1050600000277800F00F200000277800F0FF2F00C5
:1050700035EF0700B8EF070037F0070002003700F0
:105080003E0078003E007800000006005600000058
:10509000CE5445004C4543004841520047454D0021
:1050A000454E54000027780080BB20008EEE07009C
:1050B000C7EC07000000060016000000C9444500C8
:1050C0004D4152005241470045000000A08A200097
:1050D00020A0B7000F8020000E9020000E00780066
:1050E0007F0509000018EB00002778001000200061
:1050F000FDEE0700B6EC070000277800800F2100C6
:1051000024F0070000277800F0FF270084EE070056
:105110008000B000AEEC070027FF0700F6F20700A2
:1051200000277800000020000027780000102000F1
:1051300063EF070057EC070056EC070000277800E4
:10514000000020000027780020002000AFEC0700BE
:1051500050EC07004FEC070059EF0700801F780064
:105160003E00780000277800F00F2000EFEC0700E9
:10517000002778004F00780000277800F0FF2F000C
:10518000EAEC07003E0060000000B0003E0078003E
:10519000EAFF32003FEC07003EEC0700F8EE0700A4
:1051A0003CEC0700002778005000200047EC070087
:1051B000DEEC070037EC07000027780050002000E5
:1051C00042EC0700D9EC07003E0060000000B00090
:1051D0003E007800050032003E0078003E00780076
:1051E00000277800F0FF2F006900370029EC070046
:1051F00028EC070000277800000020000027780036
:105200002000200093EC07002DEF070021EC0700A1
:105210000000B0003E0078000A0032003E00780036
:105220003E0078000027780000002000002778006A
:105230002000200087EC07000027780000002000F5
:1052400053003700801F78003E007800801F7800F0
:105250003E0078000FEC07000EEC070000277800F6
:105260004F007800002778004F00780079EC0700A5
:1052700008EC07004F80DE000000B0003E00780020
:105280000C0032003E0078003E00780000277800D5
:105290000000200000277800200020006DEC0700AF
:1052A000002778000000200000277800F0FF2F0082
:1052B00034003700F7EB070000277800700020006B
:1052C00002EC070099EC0700F2EB070000277800DA
:1052D00070002000FDEB070094EC07003E0060002A
:1052E0000000B0003E0078000A0032003E00780066
:1052F0003E007800EDEB07003E007800EBEB070086
:105300003E00780000277800F0FF2F00002778008B
:105310001C003700DFEB0700DEEB070000277800FA
:1053200000002000002778002000200049EC070042
:10533000E3EE0700D7EB07000000B0003E00780066
:105340000E0032003E0078003E0078003E007800FB
:105350003E00780000277800000020000027780039
:10536000200020003BEC0700002778000000200010
:1053700000277800F0FF2F00020037000027780098
:10538000000020000000B0003E007800B7FF3200AF
:105390000000B0003E00780081FF3200BDEB070046
:1053A000BCEB070008EE070000277800801F78009C
:1053B0003E00780006EC0700002778004F007800D8
:1053C0002000B00002EC0700B2EB0700B1EB0700D1
:1053D000BBEE0700801F78003E00780000277800B1
:1053E0001004200051EC0700002778004F007800DF
:1053F0000027780050CC24004CEC07003E006000F1
:105400000000B0003E007800200032000027780045
:10541000000020000027780020002000FBEB0700A0
:105420009CEB07009BEB0700A5EE0700801F7800B0
:105430003E00780000277800500420003BEC070075
:10544000002778004F00780000277800E03424001F
:1054500036EC07003E0060000000B0003E0078001F
:1054600007003200002778000000200000277800A5
:1054700020002000E5EB0700FCF6070002003700E3
:105480003E0078003E007800020037003E007800C1
:105490003E00780010F207008AFE070016F10700B0
:1054A00048FB070000000600FFFFFF00FFFFFF00B2
:00000001FF
